:100000000C94D9000C94F4000C94F4000C94F400BB
:100010000C94F4000C94F4000C9409160C94F40065
:100020000C94F4000C94F4000C948E160C944F165F
:100030000C940D110C94F4000C94F4000C94F40046
:100040000C94F4000C9402040C94F4000C94CE0F65
:100050000C9421100C94F4000C94F4000C94F40013
:100060000C94F4000C94F4000C94F4000C94F40040
:100070004570692D4F5344205665722E302E382E10
:1000800031610000416B7475656C6C65732053655C
:100090007474696E67000053657474696E6720201C
:1000A0000000486F6568656E73656E736F7220003F
:1000B000004853206D697420536368616C746572E5
:1000C00020000048656164696E6720486F6C642099
:1000D00000004B6F6D706173732000004B6F6D708B
:1000E0006173732066697820000047505320416B8C
:1000F00074697620000041636873656E6B6F707081
:10010000656C756E67200000447265687261746585
:1001100020626567722E2000004665686C6572205B
:1001200046433C2D3E4F53442000004B65696E65AD
:100130002053657474696E672D416E7A65696765D1
:10014000000050432F4254206973742065696E6724
:1001500065736368616C7465740000DC6265726E5F
:1001600065686D65204C65747A7465732053657499
:1001700074696E6700004F4E00002D2D2D00004564
:1001800050492D4D656E750050616C0050432F42F3
:1001900054004B656E6E756E670052432D42657458
:1001A00072696562000045786974004F4E002D2D1C
:1001B000000011241FBECFEFD4E0DEBFCDBF11E0A1
:1001C000A0E0B1E0E2E7FEE202C005900D92AC349F
:1001D000B107D9F713E0ACE4B1E001C01D92AF372D
:1001E000B107E1F70C9401010C94000080E981BB98
:1001F0008FE084BBAC9AAD9A8EE28ABBD99ADD9A25
:1002000008951F9310928E0110928A0110928F010F
:10021000A0E0B0E00E942517802D9927809353011C
:10022000A1E0B0E00E942517802D9927809300015E
:10023000A2E0B0E00E942517802D992780935401F9
:10024000A7E1B0E00E942517802D992780936601D1
:10025000A8E1B0E00E942517802D992780937901AD
:100260000E94AE150E94F6000E94F2038091530195
:10027000813019F40E94B90F02C00E94A90F78942E
:10028000A89A0E9488030E9463040E94F6080E94B4
:1002900072090E94FE0880914E01813071F4109223
:1002A0004E0180918E01882311F40E94C3100E9498
:1002B00000110E9405110E94AA1380915201909191
:1002C0008E01813041F4992331F40E942B0F0E945A
:1002D00035130E949112809151018130E9F580918E
:1002E0008E018823C9F5AA9A0E94620E8091660148
:1002F0008823C9F40E94C8070E94B806809179013A
:1003000080FF04C00E9480110E94D2090E941D0833
:100310000E9422098091790183FF02C00E94A50BEF
:100320000E94B50918C080910201823064F00E94D9
:100330001D080E9422090E9480110E94D2090E9479
:10034000A50B0E94B50980910201833024F00E9420
:10035000C8070E94B806AA9880914C018130B1F577
:1003600080918E01882391F510924C018091660155
:10037000882321F080910201833014F00E94FE084E
:100380008091630190916401019690936401809340
:1003900063018091630190916401CC9769F480912D
:1003A00061019091620101969093620180936101D5
:1003B00010926401109263010E94070C0E94600970
:1003C00080915901813011F40E94BB0C10914D01B4
:1003D000113009F060CF80918E01882309F05BCF46
:1003E00010924D0180917F01813019F0823059F4D3
:1003F00006C00E94CD0982E080937F0104C00E9464
:10040000B00910937F0180916601813009F043CFDC
:1004100080918E01882309F03ECF80916501813063
:1004200009F039CF1092650180910201813071F09D
:1004300082301CF4882339F02ECF823081F0833053
:1004400009F029CF17C00E94CD0925CF0E94B0091D
:1004500064E084E00E9441020E9464041CCF0E9478
:10046000B00964E084E00E9441020E94F6080E9404
:10047000720911CF0E94B00964E084E00E94410239
:1004800004CF482FD99827E030E0DB980000000027
:100490000000000081E090E0022E02C0880F991F4A
:1004A0000A94E2F7842311F0DA9A01C0DA98000086
:1004B000000000000000DB9A0000000000000000C7
:1004C000215030408FEF2F3F3807F9F627E030E01A
:1004D000DB98000000000000000081E090E0022EA8
:1004E00002C0880F991F0A94E2F7862311F0DA9A66
:1004F00001C0DA980000000000000000DB9A000054
:10050000000000000000215030408FEF2F3F3807DF
:10051000F9F6DB98DA98D99A089564E084E00E94AD
:1005200041026CE480E00E94410210924E018091F1
:100530004E018823E1F36AE08CE60E94410260E00C
:1005400085E00E94410208951F93CF93DF9380912D
:100550004C018823E1F310924C010E94751010E0C9
:100560000DC080915101813011F40E94620E809182
:100570004C01813019F410924C0111E090917A01F4
:1005800080E0112309F481E0992311F4882349F7CD
:10059000C8E1D0E0882309F4A4C080916A03809365
:1005A000790180917901DE01082E0E942D1744E81F
:1005B00050E062E082E00E94490B47E950E064E0CD
:1005C00082E00E94490B42EA50E066E082E00E942D
:1005D000490B41EB50E067E082E00E94490B43EC9D
:1005E00050E068E082E00E94490B42ED50E069E093
:1005F00082E00E94490B4CED50E06AE082E00E94EC
:10060000490B4AEE50E06BE082E00E94490B46EF56
:1006100050E06CE082E00E94490B409177015091DC
:10062000780164E084E10E941E0B8091790180FFD3
:1006300003C046E751E002C04AE751E066E084E1CA
:100640000E94490B8091790181FF03C046E751E088
:1006500002C04AE751E067E084E10E94490B8091C3
:10066000790182FF03C046E751E002C04AE751E04A
:1006700068E084E10E94490B8091790183FF03C007
:1006800046E751E002C04AE751E069E084E10E9498
:10069000490B8091790184FF03C046E751E002C015
:1006A0004AE751E06AE084E10E94490B80917901B8
:1006B00085FF03C046E751E002C04AE751E06BE026
:1006C00084E10E94490B8091790186FF03C046E7CF
:1006D00051E002C04AE751E06CE084E10E94490B1E
:1006E00013C044E850E062E082E00E94490B49E117
:1006F00051E065E082E00E94490BDE010E9425176F
:10070000802D992780937901DF91CF911F910895D2
:100710000E948D0210924C0180914C018823E1F3DC
:1007200040E750E062E087E00E94490B0E946404C9
:1007300010924C0180914C018823E1F310924C01FE
:1007400080914C018823E1F310924C0164E084E035
:100750000E9441026CE480E00E94410280915301BA
:10076000882319F40E94A4021AC04BE251E062E00F
:1007700082E00E94490B42E451E064E082E00E9482
:10078000490B4BE551E066E082E00E94490BA8E18D
:10079000B0E00E942517802D9927809379018091E0
:1007A0004C018823E1F310924C0180914C01882385
:1007B000E1F310924C0180914C018823E1F31092F7
:1007C0004C0180914C018823E1F310924C018091FF
:1007D0004C018823E1F310924C0164E084E00E9414
:1007E0004102089582E083BF92E49EBD8EE189BFFD
:1007F00083E087BD86E982BD90938A0080E2809382
:100800007D0008951F920F920FB60F9211248F93BF
:100810009F93809150018F5F809350018091500190
:10082000883439F591E090934F01109250018091F6
:1008300077038F5F8093770380917703843631F459
:100840001092770390934C0190934D018091770320
:10085000823311F490934D01809176038F5F8093E2
:100860007603809176038A3021F410927603909378
:100870004E019F918F910F900FBE0F901F90189572
:10088000282F80538A3010F090E005C0203311F4F7
:100890009AE001C0982F822F81548A3110F4922F50
:1008A0009653822F81568A3110F4922F9C532D3209
:1008B00011F499E403C02E3209F491E4892F9927A9
:1008C00087FD90950895089560E085E00E944102BB
:1008D00063E886E00E94410260E987E00E944102ED
:1008E00060E085E00E94410264E886E00E944102E7
:1008F00061E987E00E94410260E085E00E944102D8
:1009000065E886E00E94410262E987E00E944102B8
:1009100060E085E00E94410266E886E00E944102B4
:1009200063E987E00E94410260E085E00E944102A5
:1009300067E886E00E94410264E987E00E94410284
:1009400060E085E00E94410268E886E00E94410282
:1009500065E987E00E94410260E085E00E94410273
:1009600069E886E00E94410266E987E00E94410250
:1009700060E085E00E9441026AE886E00E94410250
:1009800067E987E00E94410260E085E00E94410241
:1009900061EA86E00E94410268E987E00E94410224
:1009A00060E085E00E94410262EA86E00E94410226
:1009B00069E987E00E94410260E085E00E9441020F
:1009C00063EA86E00E9441026AE987E00E944102F0
:1009D00060E085E00E94410264EA86E00E944102F4
:1009E0006BE987E00E94410260E085E00E944102DD
:1009F00065EA86E00E9441026CE987E00E944102BC
:100A000060E085E00E94410266EA86E00E944102C1
:100A10006DE987E00E94410260E085E00E944102AA
:100A200067EA86E00E9441026EE987E00E94410287
:100A300060E085E00E94410268EA86E00E9441028F
:100A40006FE987E00E94410260E085E00E94410278
:100A50006FEB86E00E94410260EA87E00E9441025B
:100A600060E085E00E94410260EC86E00E94410265
:100A700061EA87E00E94410260E085E00E94410255
:100A800061EC86E00E94410262EA87E00E94410236
:100A900060E085E00E94410262EC86E00E94410233
:100AA00063EA87E00E94410260E085E00E94410223
:100AB00063EC86E00E94410264EA87E00E94410202
:100AC00060E085E00E94410264EC86E00E94410201
:100AD00065EA87E00E94410260E085E00E944102F1
:100AE00065EC86E00E94410266EA87E00E944102CE
:100AF00060E085E00E94410266EC86E00E944102CF
:100B000067EA87E00E94410260E085E00E944102BE
:100B10006DED86E00E94410268EA87E00E94410292
:100B200060E085E00E9441026EED86E00E94410295
:100B300069EA87E00E94410260E085E00E9441028C
:100B40006FED86E00E9441026AEA87E00E9441025E
:100B500060E085E00E94410260EE86E00E94410272
:100B60006BEA87E00E94410260E085E00E9441025A
:100B700061EE86E00E9441026CEA87E00E94410239
:100B800060E085E00E94410262EE86E00E94410240
:100B90006DEA87E00E94410260E085E00E94410228
:100BA00063EE86E00E9441026EEA87E00E94410205
:100BB00060E085E00E94410264EE86E00E9441020E
:100BC0006FEA87E00E94410260E085E00E944102F6
:100BD0006BEF86E00E94410260EB87E00E944102D9
:100BE00060E085E00E9441026CEF86E00E944102D5
:100BF00061EB87E00E94410260E085E00E944102D3
:100C00006DEF86E00E94410262EB87E00E944102A4
:100C100060E085E00E9441026EEF86E00E944102A2
:100C200063EB87E00E94410260E085E00E944102A0
:100C30006FEF86E00E94410264EB87E00E94410270
:100C400061E085E00E94410260E086E00E9441028E
:100C500065EB87E00E94410261E085E00E9441026D
:100C600061E086E00E94410266EB87E00E9441025B
:100C70000895FF920F931F93CF93DF938C01F62E6D
:100C8000EC0117C06D2F772785E00E9441026C2F81
:100C900086E00E9441028F2D9927FC01EE0FFF1F75
:100CA000E80FF91FE15FFE4F608187E00E9441027B
:100CB0002196C8010596C817D90720F3E8012A969E
:100CC00017C06D2F772785E00E9441026C2F86E0C8
:100CD0000E9441028F2D9927FC01EE0FFF1FE80FA4
:100CE000F91FE15FFE4F608187E00E94410221967B
:100CF000C8010F96C817D90720F3DF91CF911F9134
:100D00000F91FF9008950F931F93CF93DF938C0162
:100D1000EC010EC06D2F772785E00E9441026C2FF9
:100D200086E00E94410260E087E00E944102219635
:100D3000C8010596C817D90768F3E8012A960EC0BE
:100D40006D2F772785E00E9441026C2F86E00E947C
:100D5000410260E087E00E9441022196C8010F969F
:100D6000C817D90768F3DF91CF911F910F910895AC
:100D70001F93CF93DF9380911E0390911F0366E131
:100D800070E00E9412179B012E5F3F4F37FD1BC082
:100D9000C9016AE070E00E941217182F1695C90168
:100DA0006AE070E00E94121787E090E0861B9109CC
:100DB0002EE130E0829FE001839FD00D929FD00D05
:100DC0001124279616C0309521953F4FC9016AE03E
:100DD00070E00E941217182F16951C5FC9016AE077
:100DE00070E00E9412178EE1689FE0011124C95043
:100DF000DF4F80910B0190910C01C817D90739F092
:100E000080910B0190910C010E94830604C0809197
:100E10007D01811721F0612FCE010E9439061093C8
:100E20007D01D0930C01C0930B01DF91CF911F91F5
:100E30000895AF92BF92DF92EF92FF920F931F93AC
:100E4000CF93DF93CDB7DEB721970FB6F894DEBF0F
:100E50000FBECDBF8C01D62E5C0119826B2D77277A
:100E600085E00E9441026A2D86E00E944102ED2C3D
:100E7000FF24F701E35DFE4F608187E00E9441029D
:100E80008EE190E0A80EB91E9981925E99839C3301
:100E900029F7F4EBAF2EB12CA00EB11E6B2D7727E6
:100EA00085E00E9441026A2D86E00E944102F7011E
:100EB000E35DFE4F608187E00E944102EEE1F0E0D9
:100EC000AE0EBF1EC801825F9E4FA816B90631F74D
:100ED00021960FB6F894DEBF0FBECDBFDF91CF9144
:100EE0001F910F91FF90EF90DF90BF90AF9008950A
:100EF000EF92FF920F931F93CF93DF93CDB7DEB79F
:100F000021970FB6F894DEBF0FBECDBF8C017C01D8
:100F100019826F2D772785E00E9441026E2D86E0B1
:100F20000E94410260E087E00E9441028EE190E071
:100F3000E80EF91E9981925E99839C3351F784EBF8
:100F4000E82EF12CE00EF11E6F2D772785E00E9430
:100F500041026E2D86E00E94410260E087E00E941F
:100F60004102EEE1F0E0EE0EFF1EC801825F9E4FEF
:100F7000E816F90649F721960FB6F894DEBF0FBEC2
:100F8000CDBFDF91CF911F910F91FF90EF9008950A
:100F90001F93CF93DF93809120039091210366E10B
:100FA00070E00E9412179B012A5F3F4F37FD12C06D
:100FB000C9016AE070E00E941217182F16951C5F95
:100FC000C9016AE070E00E941217C6E8D0E0C61BB3
:100FD000D10913C0309521953F4FC9016AE070E0F7
:100FE0000E941217182F1695C9016AE070E00E943E
:100FF0001217C62FDD27C957DF4F80910D01909141
:101000000E01C817D90739F080910D0190910E019A
:101010000E94780704C080917E01811721F0612F22
:10102000CE010E94190710937E01D0930E01C09348
:101030000D01DF91CF911F910895FF920F931F93A0
:10104000CF93DF9380913003909131038E55904080
:1010500063E070E00E941217EB016A3071051CF02A
:10106000C9E0D0E004C077FF02C0C0E0D0E08091CA
:101070005F0190916001C817D90709F47DC0C230A3
:10108000D10514F468E101C068E084E00E944102E7
:10109000D0936001C0935F01C530D105B9F1C6306E
:1010A000D1057CF4C230D10521F1C330D1051CF447
:1010B0002197A9F419C0C330D10501F1249779F41F
:1010C00021C0C730D10549F1C730D1051CF1C83066
:1010D000D10531F1299719F4BBE8FB2E23C0A8E80C
:1010E000FA2E04E810E820C0F8E8FF2E04E811E822
:1010F0001BC0E8E8FE2E04E812E816C078E8F72ED8
:1011000004E811C068E8F62E05E80DC058E8F52E91
:1011100006E809C048E8F42E05C039E8F32E02C0FD
:101120002AE8F22E07E813E860E085E00E94410219
:101130006FE186E00E944102612F87E00E94410238
:1011400060E085E00E9441026DE386E00E9441027A
:10115000602F87E00E94410260E085E00E9441022A
:101160006BE586E00E9441026F2D87E00E944102FC
:1011700060E084E00E944102DF91CF911F910F91C6
:10118000FF900895EF92FF920F931F93CF93DF93F9
:101190007A019EE1699FB0011124680F711D8B01D6
:1011A000020F111D10927803EB0116C06D2F7727E7
:1011B00085E00E9441026C2F86E00E9441028091EE
:1011C0007803F701E80FF11D60818F5F809378034A
:1011D00087E00E9441022196C017D10738F3DF91C2
:1011E000CF911F910F91FF90EF90089525E046E079
:1011F00051E06EE081E00E94C2080895CF93DF9332
:10120000CDB7DEB725970FB6F894DEBF0FBECDBFC2
:10121000DE011196EAE3F1E085E001900D92815044
:10122000E1F725E0AE014F5F5F4F67E08CE00E9481
:10123000C20825960FB6F894DEBF0FBECDBFDF9172
:10124000CF910895CF93DF93CDB7DEB724970FB634
:10125000F894DEBF0FBECDBF19821A8285E48B835E
:101260001C8230913003832F6AE00E94F216282FEF
:101270000E94F216482F822F0E94F216292F832FE8
:101280000E94F216992319F48AE08C8301C09C8392
:10129000222319F48AE08A8301C02A83498324E047
:1012A000AE014F5F5F4F62E083E00E94C208249668
:1012B0000FB6F894DEBF0FBECDBFDF91CF9108957A
:1012C00080915401813069F420919701922F27FD7C
:1012D0009F5F959548E951E061E08EE0891B0E948F
:1012E000C208089560E085E00E9441026FE186E057
:1012F0000E94410260E887E00E94410260E085E0D0
:101300000E9441026DE386E00E94410264E887E0AA
:101310000E94410260E085E00E9441026BE586E0A8
:101320000E94410268E887E00E944102089560E05F
:1013300085E00E9441026FEC86E00E9441026CE869
:1013400087E00E94410261E085E00E9441026BE07B
:1013500086E00E9441026DE887E00E944102089504
:101360006CE480E00E9441020895809132039091E4
:101370003303843B910544F480917F01882361F419
:1013800081E080937F01089580917F01181614F405
:101390000E94B00910927F01089562E480E00E94EB
:1013A00041020895EF92FF920F931F93CF93DF9323
:1013B000CDB7DEB72F970FB6F894DEBF0FBECDBF07
:1013C00085E0FE01369611928A95E9F7809128030F
:1013D000909129036EE170E00E941217CB018E01FB
:1013E000055F1F4F019797FF02C080E090E04AE041
:1013F00050E0B8010E94C116F80101900020E9F701
:101400003197EE2EE01A10927803FF240AC00E0FD7
:101410001F1FEC0FFD1F83850E944004F80180838D
:10142000F394EF2DFF278E2D992787FD90958E0140
:101430000F5F1F4FE817F90754F3F092780325E088
:10144000AE014A5F5F4F69E085E10E94C2082E2D20
:10145000A80169E089E18E190E94C2082F960FB693
:10146000F894DEBF0FBECDBFDF91CF911F910F91DA
:10147000FF90EF900895EF92FF920F931F93CF93F9
:10148000DF93CDB7DEB72E970FB6F894DEBF0FBE51
:10149000CDBF19821A821B821C8280916F019091AC
:1014A00070018E01065F1F4F4AE050E0B8010E94B4
:1014B000C116F80101900020E9F73197EE2EE01AED
:1014C00010927803FF240AC00E0F1F1FEC0FFD1FA0
:1014D00082850E944004F8018083F394EF2DFF275A
:1014E0008E2D992787FD90958E010B5F1F4FE81772
:1014F000F90754F3F092780324E0AE014F5F5F4F99
:1015000066E085E10E94C2082E2DA80166E089E10F
:101510008E190E94C20880916F0190917001181677
:10152000190664F460E085E00E94410262EC86E006
:101530000E9441026CE887E00E94410280916F01A5
:101540009091700197FF0CC060E085E00E9441021D
:1015500062EC86E00E9441026DE887E00E94410251
:1015600080916F0190917001892B61F460E085E0BA
:101570000E94410262EC86E00E94410260E087E046
:101580000E9441022E960FB6F894DEBF0FBECDBF6B
:10159000DF91CF911F910F91FF90EF9008959F924F
:1015A000AF92BF92CF92DF92EF92FF920F931F9371
:1015B000CF93DF93CDB7DEB76E970FB6F894DEBF4B
:1015C0000FBECDBF982EA62E7A01FA010190002001
:1015D000E9F73197BE2EB41ACC24DD240BC0FF27C7
:1015E0008A010E0F1F1FEE0DFF1D80810E94400417
:1015F000F8018083EC2D0894C11CD11C8B2D9927F8
:101600000196AE014F5F5F4FC816D90641F72B2DEB
:101610006A2D892D0E94C2086E960FB6F894DEBF1F
:101620000FBECDBFDF91CF911F910F91FF90EF9033
:10163000DF90CF90BF90AF909F900895EF92FF9270
:101640000F931F93CF93DF93CDB7DEB764970FB699
:10165000F894DEBF0FBECDBFE82EF62ECA014AE0D9
:1016600050E08E010F5F1F4FB8010E94C116A80104
:101670006F2D8E2D0E94CF0A64960FB6F894DEBFB0
:101680000FBECDBFDF91CF911F910F91FF90EF90D3
:101690000895BF92CF92DF92EF92FF920F931F9324
:1016A000CF93DF93CDB7DEB764970FB6F894DEBF64
:1016B0000FBECDBFB82EC62E9A01DE01119605C011
:1016C000EA0FFB1F90832F5F3F4F822F841BF9018E
:1016D0009491E82FFF27992399F7EA0FFB1F1082B7
:1016E000FD0101900020E9F73197DE2EDA1AEE2491
:1016F000FF2409C08D01020F111DF80180810E9495
:101700004004F80180832E2D0894E11CF11C8D2DDE
:1017100099270196DE011196E816F90659F72D2D45
:10172000AD016C2D8B2D0E94C20864960FB6F89403
:10173000DEBF0FBECDBFDF91CF911F910F91FF9004
:10174000EF90DF90CF90BF900895EF92FF920F93AC
:101750001F93CF93DF93CDB7DEB72B970FB6F894D7
:10176000DEBF0FBECDBFDE011196E7E3F1E083E0FF
:1017700001900D928150E1F78E01085F1F4F4AE002
:1017800050E0B80180912E0390912F030E94C11662
:10179000F80101900020E9F73197EE2EE01A10923F
:1017A0007803FF240AC00E0F1F1FEC0FFD1F80855A
:1017B0000E944004F8018083F394EF2DFF278E2DC3
:1017C000992787FD90958E010C5F1F4FE817F90749
:1017D00054F3F092780323E0AE014F5F5F4F6EE069
:1017E0008DE00E94C2082E2DA8016EE080E18E19C6
:1017F0000E94C2082B960FB6F894DEBF0FBECDBF75
:10180000DF91CF911F910F91FF90EF900895EF928C
:10181000FF920F931F93CF93DF93CDB7DEB7289737
:101820000FB6F894DEBF0FBECDBF19828AE08A835F
:1018300080916101909162018E010A5F1F4F4AE021
:1018400050E0B8010E94C116F80101900020E9F7AC
:101850003197EE2EE01A10927803FF240DC08E010E
:101860000D5F1F4F0E0F1F1FEC0FFD1F86810E9483
:101870004004F8018083F394EF2DFF278E2D9927E4
:1018800087FD9095E817F90754F3F092780380915B
:101890006101909162018E010D5F1F4F0A976CF4F8
:1018A00021E0AE014F5F5F4F6EE081E00E94C20811
:1018B00021E0A8016EE082E004C022E0A8016EE011
:1018C00081E00E94C20880916301909164018E01C1
:1018D0000A5F1F4F4AE050E0B8010E94C116F801AC
:1018E00001900020E9F73197EE2EE01A109278036C
:1018F000FF240DC08E010D5F1F4F0E0F1F1FEC0F39
:10190000FD1F86810E944004F8018083F394EF2D2F
:10191000FF278E2D992787FD9095E817F90754F337
:10192000F092780380916301909164018E010D5FC4
:101930001F4F0A976CF421E0AE014E5F5F4F6EE0DF
:1019400084E00E94C20821E0A8016EE085E004C0A6
:1019500022E0A8016EE084E00E94C20828960FB63B
:10196000F894DEBF0FBECDBFDF91CF911F910F91D5
:10197000FF90EF900895CF92DF92EF92FF920F9336
:101980001F93CF93DF93CDB7DEB72B970FB6F894A5
:10199000DEBF0FBECDBF80915A0190915B0162E026
:1019A00070E00E94121770935B0160935A0180915E
:1019B0005A0190915B018456904090935B01809313
:1019C0005A0180915A0190915B0197FF04C01092D7
:1019D0005B0110925A0180915A0190915B018D5ADE
:1019E000964234F08CEA96E290935B0180935A0120
:1019F00080915A0190915B0164E670E00E94FE16AE
:101A0000709356016093550180915A0190915B014A
:101A100064E670E00E94FE1690935801809357018F
:101A200080915701909158016AE070E00E94FE1683
:101A30007093580160935701809155019091560120
:101A400025E429831A821B828E01085F1F4F4AE01A
:101A500050E0B8010E94C116F80101900020E9F79A
:101A60003197CE2EC01A10927803DD240BC0020FDE
:101A7000131FE20EF31EF70180810E944004F8015B
:101A80008083D3942D2D33278C2D992787FD909516
:101A900048E0E42EF12CEC0EFD1E8E010C5F1F4F72
:101AA0002817390724F3D092780322E0AE014E5F65
:101AB0005F4F63E083E00E94C2082C2DA80163E021
:101AC00085E08C190E94C2088091570190915801BD
:101AD0004AE050E0B7010E94C116F70101900020D2
:101AE000E9F73197EE19EE2E10927803FF240AC021
:101AF0000E0F1F1FEC0FFD1F80850E944004F80190
:101B00008083F394EF2DFF278E2D992787FD9095E5
:101B10008E010C5F1F4FE817F90754F3F09278031A
:101B200021E0AE014F5F5F4F63E085E00E94C20895
:101B300021E0AE014E5F5F4F63E086E00E94C20885
:101B400021E0A80163E086E00E94C2082B960FB650
:101B5000F894DEBF0FBECDBFDF91CF911F910F91E3
:101B6000FF90EF90DF90CF9008950F931F93CF9346
:101B7000DF93CDB7DEB72A970FB6F894DEBF0FBE5E
:101B8000CDBF4AE050E08E010F5F1F4FB8010E94A9
:101B9000C116F80101900020E9F73197E01B10927F
:101BA000780320E0FF27E7FDF09501C02F5F822F2B
:101BB00099278E179F07D4F3209378032A960FB6A0
:101BC000F894DEBF0FBECDBFDF91CF911F910F9173
:101BD0000895EF92FF920F931F93CF93DF9333E01B
:101BE000E32EF12CC0E0D0E0A9E8B2E08C91FD0139
:101BF000218112810381B7016C5F7F4F7B011496B5
:101C0000F2E0673C7F0709F456C0422F55274D5339
:101C10005040E0914301F0914401EC0FFD1F9927E2
:101C2000CD97880F991F880F991F9A01689413F810
:101C3000359527951694E1F7822B932B80836B3192
:101C40007105C9F1212F33272D533040FE01319604
:101C50008091430190914401E80FF91F4F7050703B
:101C600084E0440F551F8A95E1F7C9019595879542
:101C700095958795482B592B408381E06F367807DF
:101C8000D1F0FE0132968091430190914401E80F1A
:101C9000F91F2370307086E0220F331F8A95E1F719
:101CA000802F9927CD97282B392B2083635C724096
:101CB00011F023969BCFDF91CF911F910F91FF9051
:101CC000EF900895EF92FF920F931F93CF93DF93BE
:101CD00080918802843409F06AC033E0E32EF12C4D
:101CE00060E070E0A9E8B2E08C91FD0121811281F1
:101CF0000381E70124967E0114966134710509F48D
:101D000056C0422F55274D535040E0913F01F0916E
:101D10004001E60FF71F9927CD97880F991F880F6D
:101D2000991F9A01689413F8359527951694E1F751
:101D3000822B932B808360347105C9F1212F3327C7
:101D40002D533040FB01319680913F01909140012D
:101D5000E80FF91F4F70507084E0440F551F8A95AB
:101D6000E1F7C9019595879595958795482B592B4E
:101D70004083CB35D105D9F0FB01329680913F01EC
:101D800090914001E80FF91F2370307046E0220F58
:101D9000331F4A95E1F7802F9927CD97282B392BB0
:101DA00020836E33710519F06D5F7F4F9DCF809159
:101DB00088028C3459F481E090E09093780180930C
:101DC000770181E080937A010E94E90D8091880279
:101DD0008D3459F482E090E09093780180937701FC
:101DE00081E080937A010E94E90D809188028E340F
:101DF00059F483E090E0909378018093770181E03B
:101E000080937A010E94E90D809188028F3459F401
:101E100084E090E0909378018093770181E0809353
:101E20007A010E94E90D80918802803559F485E09D
:101E300090E0909378018093770181E080937A011C
:101E40000E94E90D10925101DF91CF911F910F91E6
:101E5000FF90EF900895EF92FF920F931F93CF930F
:101E6000DF938091AE01843409F06AC033E0E32E41
:101E7000F12C60E070E0AFEAB1E08C91FD012181CE
:101E800012810381E70124967E0114966134710565
:101E900009F456C0422F55274D535040E09141015F
:101EA000F0914201E60FF71F9927CD97880F991FF0
:101EB000880F991F9A01689413F835952795169401
:101EC000E1F7822B932B808360347105C9F1212FB8
:101ED00033272D533040FB01319680914101909181
:101EE0004201E80FF91F4F70507084E0440F551FF6
:101EF0008A95E1F7C9019595879595958795482B22
:101F0000592B4083CB35D105D9F0FB013296809116
:101F1000410190914201E80FF91F2370307046E0B3
:101F2000220F331F4A95E1F7802F9927CD97282B51
:101F3000392B20836E33710519F06D5F7F4F9DCF74
:101F400010925201DF91CF911F910F91FF90EF906E
:101F5000089582E289B910BC80B91CBE909A28E924
:101F60002AB996E890BD82EC8BB921B99CBF82B9A1
:101F7000089582E289B910BC80B91CBE909A88E9A4
:101F80008AB926E820BD92EC9BB980E981B92CBFC3
:101F900092B90895159BFECF83B908951F920F92B1
:101FA0000FB60F9211248F939F93EF93FF939CB1E1
:101FB000909379039D3081F480918101813061F4A7
:101FC000AB981092810180935201E0916103FF2749
:101FD000E455FE4F90832CC080918101882319F035
:101FE000813031F513C0933239F480915201882346
:101FF00019F481E080938101109261038091610363
:10200000E82FFF27E455FE4F90830CC0E091610359
:10201000FF27E455FE4F908380916103853930F4AA
:10202000809161038F5F8093610302C010928101F0
:10203000FF91EF919F918F910F900FBE0F901F9086
:1020400018951F920F920FB60F9211248F939F93A2
:10205000EF93FF9393B190937A039D3081F4809135
:102060008001813061F4AB9810928001809351011E
:10207000E0915E03FF27EA57FD4F90832DC08091CA
:102080008001882319F0813039F514C0933241F46E
:1020900080915101882321F481E080938001AB9AE3
:1020A00010925E0380915E03E82FFF27EA57FD4FF1
:1020B00090830CC0E0915E03FF27EA57FD4F9083A9
:1020C00080915E03853930F480915E038F5F809349
:1020D0005E0302C010928001FF91EF919F918F915A
:1020E0000F900FBE0F901F901895CF93DF93CDB731
:1020F000DEB72C970FB6F894DEBF0FBECDBF83E2DC
:1021000089831A8281E78B838CE78C838DE68D83AC
:102110008DE38E838F8320E030E0FE013196AE01A7
:10212000485F5F4F8191280F311DE417F507D1F704
:10213000C90160E070E10E9412179C0160E470E048
:102140000E941217635C6887C90160E470E00E9416
:102150001217835C89878DE08A87FE0131969E0184
:10216000255F3F4F8081159BFECF83B93196E217E3
:10217000F307C1F72C960FB6F894DEBF0FBECDBFA4
:10218000DF91CF910895CF93DF93CDB7DEB72A9734
:102190000FB6F894DEBF0FBECDBF83E289831A82EB
:1021A00083E68B831C821D8286E890E060E070E10C
:1021B0000E9412179C0160E470E00E941217635C99
:1021C0006E83C90160E470E00E941217835C8F8304
:1021D0008DE08887FE0131969E01275F3F4F808109
:1021E000159BFECF83B93196E217F307C1F72A9604
:1021F0000FB6F894DEBF0FBECDBFDF91CF9108952B
:1022000085B392E0892785BB089590915E01913056
:1022100019F485B3892785BB08951F920F920FB6D5
:102220000F9211242F933F935F936F937F938F931C
:102230009F93AF93BF938091820190918301892BEB
:1022400081F484B595B590938901809388018EB50A
:102250008F7B8EBD81E090E090938301809382011B
:1022600041C084B595B590938701809386012EB5C2
:1022700020642EBD2091880130918901821B930B2F
:102280001092830110928201865698406CE271E0B0
:102290000E94FE16709385016093840177FF05C04C
:1022A000109285011092840109C06730710534F0E5
:1022B00086E090E0909385018093840120918401D1
:1022C0003091850180910201992787FD909528170B
:1022D000390741F0263031052CF42093020181E0CA
:1022E00080936501BF91AF919F918F917F916F9185
:1022F0005F913F912F910F900FBE0F901F901895F7
:10230000809128039091290390936801809367013D
:1023100080916701909168012091690130916A0173
:10232000821B930B90936C0180936B0180916701EA
:102330009091680190936A018093690140917301C3
:102340005091740120916B0130916C01CA01E3E05E
:10235000880F991FEA95E1F7841B950B73E0220F14
:10236000331F7A95E1F7820F931F68E070E00E94B7
:10237000121770937401609373012091750130916D
:1023800076014091730150917401C90163E0880F97
:10239000991F6A95E1F7821B930B840F951F68E0E4
:1023A00070E00E941217709376016093750180911E
:1023B0007501909176019093700180936F010E9456
:1023C0003B0A0895BF92CF92DF92EF92FF920F9354
:1023D0001F93CF93DF93CDB7DEB760970FB6F89416
:1023E000DEBF0FBECDBF19821A821B821C82809174
:1023F0007A0290917B0290937E0380937D0380917B
:102400007C0290917D0290937C0380937B0380916A
:102410007D0390917E038E01055F1F4F4AE050E0DF
:10242000B8010E94C116F80101900020E9F7319728
:10243000BE2EB01ACC24DD240DC0EC0CFD1CF7011F
:1024400080810E9440040C0D1D1DF80180830894BA
:10245000C11CD11C8B2D992787FD90952BE0E22E76
:10246000F12CEC0EFD1E8E010B5F1F4FC816D90616
:1024700024F324E0AE014F5F5F4F61E08CE00E94E7
:10248000C2082B2DA80161E080E18B190E94C208CF
:1024900080917B0390917C034AE050E0B7010E9459
:1024A000C116F70101900020E9F73197DE2EDE1802
:1024B000EE24FF240DC0FE01EE0DFF1D83850E945A
:1024C00040040E0D1F1DF80180830894E11CF11CCF
:1024D0008D2D992787FD90958E010B5F1F4FE81674
:1024E000F9064CF324E0AE014F5F5F4F62E08CE0F1
:1024F0000E94C2082D2DA80162E080E18D190E9482
:10250000C20860960FB6F894DEBF0FBECDBFDF9154
:10251000CF911F910F91FF90EF90DF90CF90BF90E0
:1025200008958F929F92BF92CF92DF92EF92FF9287
:102530000F931F93CF93DF93CDB7DEB760970FB69E
:10254000F894DEBF0FBECDBF19821A821B821C8297
:1025500080904203909043038E01055F1F4F4AE035
:1025600050E0B80180914003909141030E94C11650
:10257000F80101900020E9F73197BE2EB01ACC2463
:10258000DD240DC0EC0CFD1CF70180810E9440048D
:102590000C0D1D1DF80180830894C11CD11C8B2DCE
:1025A000992787FD90953BE0E32EF12CEC0EFD1E64
:1025B0008E010B5F1F4FC816D90624F324E0AE012D
:1025C0004F5F5F4F64E08CE00E94C2082B2DA80192
:1025D00064E080E18B190E94C2084AE050E0B70134
:1025E000C4010E94C116F70101900020E9F731975C
:1025F000DE2EDE18EE24FF240DC0FE01EE0DFF1DC1
:1026000083850E9440040E0D1F1DF80180830894ED
:10261000E11CF11C8D2D992787FD90958E010B5F94
:102620001F4FE816F9064CF324E0AE014F5F5F4FF1
:1026300065E08CE00E94C2082D2DA80165E080E1D4
:102640008D190E94C20860960FB6F894DEBF0FBEC7
:10265000CDBFDF91CF911F910F91FF90EF90DF9051
:10266000CF90BF909F908F900895DF92EF92FF924E
:102670000F931F93CF93DF93CDB7DEB72B970FB692
:10268000F894DEBF0FBECDBFDE011196E9E4F1E0A4
:1026900083E001900D928150E1F78E01085F1F4F9A
:1026A0004AE050E0B80180918202909183020E943A
:1026B000C116F80101900020E9F73197DE2ED01AFB
:1026C000EE24FF240DC0FE01EE0DFF1D80850E944B
:1026D00040040E0D1F1DF80180830894E11CF11CBD
:1026E0008D2D992787FD90958E010C5F1F4FE81661
:1026F000F9064CF323E0AE014F5F5F4F61E088E1E4
:102700000E94C2082D2DA80161E08BE18D190E9465
:10271000C2082B960FB6F894DEBF0FBECDBFDF9177
:10272000CF911F910F91FF90EF90DF90089522E0DD
:1027300047E451E061E08AE10E94C2080895F894FC
:1027400088E190E028E00FB6F894A89581BD0FBE0F
:1027500021BDFFCF1F939D9902C180918A018F5F98
:1027600080938A0191E090938C0180918A01853059
:1027700009F0F9C080918E01882309F071C090930F
:102780008E0110928F0164E084E00E94410220914A
:10279000970148E951E061E083E00E94C2084FE7F9
:1027A00051E063E083E00E94490B68E084E00E940E
:1027B000410248E851E065E083E00E94490B8091C6
:1027C0000001813019F44BEA51E002C04EEA51E0B9
:1027D00065E084E10E94490B60E084E00E944102D0
:1027E0004CE851E066E083E00E94490B8091530180
:1027F000813019F44BEA51E002C04EEA51E066E044
:1028000084E10E94490B42E951E067E083E00E94C5
:10281000490B80915401813019F44BEA51E002C018
:102820004EEA51E067E084E10E94490B4AE951E039
:1028300068E083E00E94490B80916601813019F4C1
:102840004BEA51E002C04EEA51E068E084E10E94A8
:10285000490B46EA51E06BE083E00E94490B81C0DE
:1028600010918F01113001F568E084E00E9441026F
:1028700080915301882329F4109353014BEA51E0CE
:1028800004C0109253014EEA51E066E084E10E94D8
:10289000490B80915301A0E0B0E0082E0E942D1753
:1028A00060E084E00E94410280918F01823009F54E
:1028B00068E084E00E94410280915401882331F451
:1028C00081E0809354014BEA51E004C0109254011E
:1028D0004EEA51E067E084E10E94490B8091540187
:1028E000A2E0B0E0082E0E942D1760E084E00E9474
:1028F000410280918F01833009F568E084E00E94F5
:10290000410280916601882331F481E08093660161
:102910004BEA51E004C0109266014EEA51E068E0D3
:1029200084E10E94490B80916601A7E1B0E0082E86
:102930000E942D1760E084E00E94410280918F0187
:10294000843089F410928E01F89488E190E028E0B8
:102950000FB6F894A89581BD0FBE21BDFFCF109290
:102960008A0110928C019C99E9C090918E0191305E
:1029700009F0EAC090938D0180918B018F5F809365
:102980008B0180918B01853009F0DEC010928B01A4
:1029900080918F01823009F464C0833030F4882341
:1029A00059F0813009F0D0C031C0833009F483C0C0
:1029B000843009F0C9C09EC090938F0148E851E06F
:1029C00065E083E00E94490B80910001813019F499
:1029D0004BEA51E002C04EEA51E065E084E10E941A
:1029E000490B68E084E00E9441024CE851E066E057
:1029F00083E00E94490B80915301813019F44BEA26
:102A000051E002C04EEA51E066E090C082E080935F
:102A10008F014CE851E066E083E00E94490B809111
:102A20005301813019F44BEA51E002C04EEA51E003
:102A300066E084E10E94490B68E084E00E94410264
:102A400042E951E067E083E00E94490B8091540124
:102A5000813019F44BEA51E002C04EEA51E067E0E0
:102A600065C083E080938F0142E951E067E00E94F6
:102A7000490B80915401813019F44BEA51E002C0B6
:102A80004EEA51E067E084E10E94490B68E084E08F
:102A90000E9441024AE951E068E083E00E94490B4C
:102AA00080916601813019F44BEA51E002C04EEA90
:102AB00051E068E03BC084E080938F014AE951E037
:102AC00068E083E00E94490B80916601813019F42F
:102AD0004BEA51E002C04EEA51E068E084E10E9416
:102AE000490B68E084E00E94410246EA51E06BE055
:102AF00083E01DC010928F0146EA51E06BE083E055
:102B00000E94490B68E084E00E94410248E851E0DD
:102B100065E083E00E94490B80910001813019F447
:102B20004BEA51E002C04EEA51E065E084E10E94C8
:102B3000490B60E084E00E94410206C010928B01C4
:102B400080918C0180918D011F910895813029F42D
:102B5000A0E0B0E0062E0E942D170895EF92FF929C
:102B60000F931F93CF93DF93CDB7DEB764970FB664
:102B7000F894DEBF0FBECDBF40E050E08E010F5F86
:102B80001F4F842F9927DC01AD5FBF4F0E9425178F
:102B9000202D3327F801E80FF91F20832223F1F0BD
:102BA0004F5F5F4F2F3F69F7108218C0FE01E00FA3
:102BB000F11F81810E94400408561E4FF801808356
:102BC0000E2D11270894E11CF11C80919701992783
:102BD00087FD9095081719074CF30EC0DE0111967A
:102BE000FD0101900020E9F73197EA1BFB0BE09310
:102BF0009701EE24FF24E4CF64960FB6F894DEBF6D
:102C00000FBECDBFDF91CF911F910F91FF90EF903D
:102C100008951F920F920FB60F9211242F933F9396
:102C20008F939F9321E020935901809190018823F5
:102C300081F4809180009091810090939201809323
:102C4000910180918A008F7B80938A00209390016C
:102C50001DC0809180009091810090935B018093D2
:102C60005A0180918A00806480938A0010929001BA
:102C700080915A0190915B012091910130919201D4
:102C8000821B930B90935B0180935A019F918F91CC
:102C90003F912F910F900FBE0F901F9018951F928C
:102CA0000F920FB60F9211248F939F9380919601EC
:102CB0008130A1F0813018F0823049F525C0809133
:102CC00094018E3129F41092940181E08093960151
:102CD000809194018F5F8093940119C09091950128
:102CE000923061F41092950180919301813019F432
:102CF0009093960103C083E08093960180919501A3
:102D00008F5F8093950103C083E0809396019F912C
:102D10008F910F900FBE0F901F9018951F920F92DA
:102D20000FB60F9211248F9380919601833011F486
:102D3000109296018F910F900FBE0F901F901895D3
:102D400080911E0390911F0365E070E00E941217AE
:102D500066507F4F77FD0FC081E0653F78071CF01C
:102D600064EF71E003C06B3F71053CF06A5F81E086
:102D70008093930104C060E070E01092930162BD03
:102D80000895FB019F01E8944230C4F04532B4F449
:102D90004A3029F497FB1EF4909581959F4F642F3C
:102DA00077270E94FE16805D8A330CF0895D81933F
:102DB000CB010097A1F716F45DE251931082C9018F
:102DC0000C94E216DC01FC0101900020E9F7329737
:102DD000AE17BF0730F47C916081708331976D939B
:102DE000F7CF0895991B79E004C0991F961708F052
:102DF000961B881F7A95C9F780950895AA1BBB1B5F
:102E000051E107C0AA1FBB1FA617B70710F0A61BEA
:102E1000B70B881F991F5A95A9F780959095BC010B
:102E2000CD01089597FB092E07260AD077FD04D01F
:102E3000E5DF06D000201AF4709561957F4F089564
:102E4000F6F7909581959F4F0895E199FECFBFBB0E
:102E5000AEBBE09A11960DB20895E199FECFBFBBCB
:102E6000AEBB0DBA11960FB6F894E29AE19A0FBE76
:022E70000895C3
:102E720001010200000A0000440000230023005464
:102E82006466536365526200516100506000506095
:102E92000051610052620053636554646667686959
:102EA2006A6B6B6A69686700000053536353531C73
:0C2EB20003420262030D0A0A1D0000002A
:00000001FF
